:100000000C94DE060C9416070C9416070C94160735
:100010000C9416070C9416070C9416070C941607EC
:100020000C9416070C9416070C94AE250C946A25B4
:100030000C9401270C9416070C9416070C941607C1
:100040000C9416070C9416070C9416070C941607BC
:100050000C9416070C94DD260C9416070C941607C6
:100060000C9416070C9416070C9416070C9416079C
:100070000C9416070C9416070C9416070C9416078C
:100080000C9416070C9416070C9416070C9416077C
:100090000C9416070C9416070C9416070C9416076C
:1000A0000C9416070C9416070C9416070763423637
:1000B000B79BD8A71A39685618AEBAAB558C1D3CF9
:1000C000B7CC5763BD6DEDFD753EF6177231BF00BD
:1000D0000000803F05A84CCDB2D44EB93836A902F5
:1000E0000C50B9918688083CA6AAAA2ABE00000036
:1000F000803F0631FF0974A1010975150026FF0034
:100100009520750881020976150026FF0095207557
:10011000089102C005010980A101850319012AB7D0
:1001200000150126B700950175108100C0050C0966
:1001300001A101850419012AA002150126A002953A
:100140000175108100C005010906A101050719E02C
:1001500029E71500250195087501810295017508AB
:1001600081010507190029FF150026FF0095067576
:100170000881000508190129059505750191029569
:100180000175039101C068747470733A2F2F7777EB
:10019000772E6769746875622E636F6D2F6E696361
:1001A0006B6F6C61696A000DF6010014F901004380
:1001B000F6010036F6010073F9010095F4010046DE
:1001C000F3010051F30100AFF4010071F10100727D
:1001D00067626C696768742064697361626C65202A
:1001E0005B454550524F4D5D3A207267626C6967BE
:1001F00068745F636F6E6669672E656E61626C65B9
:10020000203D2025750A007267626C69676874205A
:10021000656E61626C65205B454550524F4D5D3A9D
:10022000207267626C696768745F636F6E66696786
:100230002E656E61626C65203D2025750A0072672F
:10024000626C6967687420746F67676C65205B45D2
:100250004550524F4D5D3A207267626C6967687411
:100260005F636F6E6669672E656E61626C65203DC7
:100270002025750A0044454255473A206469736158
:10028000626C65642E0A0044454255473A20656E0B
:1002900061626C65642E0A003F00433E20004F6E91
:1002A0006573686F743A206163746976653A2025D6
:1002B000640A000A002530325820006B6579626FAD
:1002C0006172645F7265706F72743A200029001465
:1002D000001A000800150017001C0018000C00127E
:1002E0000013002A002B0004001600070009000A72
:1002F000000B000D000E000F0033003100E1001D67
:10030000001B000600190005001100100036003720
:100310000052004C00E000E30001512C00000000FE
:1003200000280000000251500051004F0035001E0F
:10033000001F0020002100220023002400250026A9
:100340000027000100B35D01000100010001000170
:1003500000010001002F00300034003800010001CE
:10036000000100010001000100010001002D002E2C
:100370000001000100E20001000100010000000096
:10038000000100000001004A0001004D00B25D3A8A
:10039000003B003C003D003E003F00400041004269
:1003A0000043000100010044004500CE5CCF5CD05A
:1003B0005CD15CD25CD35CD55C0000C35C01000006
:1003C0008001800280038004800780058006800809
:1003D000800980C65C3900010001000100000000B6
:1003E00000010000000100010001000100556E69DC
:1003F000636F646520696E707574206D6F6465202D
:10040000696E697420746F3A2025750A00726762FC
:100410006C696768745F636F6E6669672E73706579
:100420006564203D2025640A007267626C69676814
:10043000745F636F6E6669672E76616C203D202560
:10044000640A007267626C696768745F636F6E66E6
:1004500069672E736174203D2025640A007267620B
:100460006C696768745F636F6E6669672E6875652F
:10047000203D2025640A007267686C696768745FB4
:10048000636F6E6669672E6D6F6465203D2025641D
:100490000A007267626C696768745F636F6E666991
:1004A000672E656E61626C65203D2025640A0072CE
:1004B00067626C696768745F636F6E666967204521
:1004C0004550524F4D3A0A007267626C6967687412
:1004D0005F696E6974207267626C696768745F63D4
:1004E0006F6E6669672E6D6F6465203D20302E202B
:1004F00057726974652064656661756C74207661F5
:100500006C75657320746F20454550524F4D2E0A0F
:10051000007267626C696768745F696E69742065F0
:1005200065636F6E666967206973206E6F742065FE
:100530006E61626C65642E0A007267626C6967683E
:10054000745F696E6974207374617274210A007239
:1005500067626C696768745F696E69742063616C57
:100560006C65642E0A007267626C69676874206447
:10057000697361626C65205B4E4F454550524F4D2B
:100580005D3A207267626C696768745F636F6E665C
:1005900069672E656E61626C65203D2025750A00D5
:1005A0007267626C6967687420656E61626C652051
:1005B0005B4E4F454550524F4D5D3A207267626C1D
:1005C000696768745F636F6E6669672E656E6162E6
:1005D0006C65203D2025750A005B735D000A0025CF
:1005E00030313662003A200025303258000A722F2E
:1005F0006320303132333435363738394142434461
:1006000045460A007F3F1F643214643214783C1E52
:100610001E140A050A0025303258006C65645F74A8
:1006200061736B3A20000001010101010101010128
:100630000202020202020202020303030303030393
:100640000304040404040404050505050506060660
:100650000606070707070708080808090909090A1D
:100660000A0A0B0B0B0C0C0C0D0D0D0E0E0E0F0FC2
:100670000F10101111111212131314141515161650
:100680001717181819191A1A1B1B1C1D1D1E1E1FBF
:100690002020212222232424252626272829292A0E
:1006A0002B2C2D2D2E2F3031323233343536373836
:1006B000393A3B3C3D3E3F40414243444546474832
:1006C000494A4C4D4E4F50515354555658595A5B08
:1006D0005D5E5F616264656668696B6C6D6F7072A8
:1006E000737577787A7B7D7E8082838587888A8C14
:1006F0008E8F91939596989A9C9EA0A2A3A5A7A948
:10070000ABADAFB1B3B5B7BABCBEC0C2C4C6C9CB3E
:10071000CDCFD1D4D6D8DBDDDFE2E4E7E9EBEEF0F4
:10072000F3F5F8FAFDFF7267626C69676874206D13
:100730006F6465205B4E4F454550524F4D5D3A20EA
:1007400025750A007267626C69676874206D6F6452
:1007500065205B454550524F4D5D3A2025750A0096
:100760007267626C69676874207365742068737659
:10077000205B4E4F454550524F4D5D3A2025752C1C
:1007800025752C25750A007267626C69676874208C
:1007900073657420687376205B454550524F4D5DFC
:1007A0003A2025752C25752C25750A007267626C18
:1007B00069676874207261696E626F77207365740F
:1007C000206873763A2025642C25642C25642C251A
:1007D000750A00FFAA7F55407267626C696768748A
:1007E0002074696D657220656E61626C65642E0AA5
:1007F000007267626C696768742074696D65722045
:1008000064697361626C652E0A00556E69636F647A
:100810006520696E707574206D6F646520736574F2
:1008200020746F3A2025750A0000000000000000C7
:1008300000000000000000000000000000000000B8
:10084000000000000000000000000000007E0F001B
:10085000D4FFFFFFC7000000780000000000000088
:10086000002A2B280000000000000000000000000B
:100870000000000029000000002C1E34202122244A
:10088000342627252E362D3738271E1F20212223D8
:100890002425263333362E37381F0405060708096A
:1008A0000A0B0C0D0E0F1011121314151617181930
:1008B0001A1B1C1D2F3130232D350405060708098E
:1008C0000A0B0C0D0E0F1011121314151617181910
:1008D0001A1B1C1D2F3130354C6B65796D61705FB3
:1008E000636F6E6669672E7261773A2025303258E1
:1008F0000A2E737761705F636F6E74726F6C5F63E3
:100900006170736C6F636B3A2025750A2E6361709A
:10091000736C6F636B5F746F5F636F6E74726F6C19
:100920003A2025750A2E737761705F6C63746C5F73
:100930006C6775693A2025750A2E737761705F724E
:1009400063746C5F726775693A2025750A2E737738
:1009500061705F6C616C745F6C6775693A202575B6
:100960000A2E737761705F72616C745F726775696C
:100970003A2025750A2E6E6F5F6775693A202575D6
:100980000A2E737761705F67726176655F65736366
:100990003A2025750A2E737761705F6261636B730D
:1009A0006C6173685F6261636B73706163653A2049
:1009B00025750A2E6E6B726F3A2025750A2E737795
:1009C00061705F6573636170655F636170736C6FA5
:1009D000636B3A2025750A0064656275675F636F13
:1009E0006E6669672E7261773A20253032580A2E7A
:1009F000656E61626C653A2025750A2E6D617472B0
:100A000069783A2025750A2E6B6579626F61726488
:100A10003A2025750A2E6D6F7573653A2025750A83
:100A2000006565636F6E6669673A0A64656661753D
:100A30006C745F6C617965723A2025750A000A0949
:100A40002D204D61676963202D0A443A094465628F
:100A50007567204D65737361676520546F67676CB8
:100A6000650A583A094D6174726978204465627567
:100A700067204D6F646520546F67676C65202D207B
:100A800053686F77206B6579707265737365732037
:100A9000696E206D617472697820677269640A4BAF
:100AA0003A094B6579626F617264204465627567CB
:100AB00020546F67676C65202D2053686F77206B1B
:100AC00065797072657373207265706F72740A4D08
:100AD0003A094465627567204D6F75736520546FE0
:100AE00067676C650A563A0956657273696F6E0AD4
:100AF000533A095374617475730A433A0941637434
:100B0000697661746520436F6E736F6C65204D6FFD
:100B100064650A46312D4631303A0953776974636A
:100B20006820746F204C6179657220302D3920283F
:100B3000463130203D204C30290A302D393A0953B6
:100B4000776974636820746F204C61796572203016
:100B50002D390A47524156453A09537769746368FB
:100B600020746F204C6179657220302028616C748C
:100B700065726E617465290A423A094A756D702082
:100B8000746F20426F6F746C6F616465720A4553B5
:100B9000433A094A756D7020746F20426F6F746C10
:100BA0006F616465722028616C7465726E61746532
:100BB000290A453A095072696E7420454550524FD2
:100BC0004D2053657474696E67730A4241434B53F9
:100BD000504143453A09436C656172204545505286
:100BE0004F4D0A000A092D20436F6E736F6C65200C
:100BF0002D0A4553432F713A09717569740A00250E
:100C000073000A092D20537461747573202D0A68CE
:100C10006F73745F6B6579626F6172645F6C65643A
:100C20007328293A20253032580A6B6579626F6142
:100C300072645F70726F746F636F6C3A202530322C
:100C4000580A6B6579626F6172645F69646C653ABA
:100C500020253032580A74696D65725F726561646F
:100C6000333228293A202530386C580A003F000AD0
:100C70006D6F7573653A206F66660A000A6D6F7551
:100C800073653A206F6E0A000A6B6579626F617254
:100C9000643A206F66660A000A6B6579626F61725A
:100CA000643A206F6E0A000A6D61747269783A20A6
:100CB0006F66660A000A6D61747269783A206F6E19
:100CC0000A000A64656275673A206F66660A000A60
:100CD00064656275673A206F6E0A000A0A4A756D8C
:100CE00070696E6720746F20626F6F746C6F6164DF
:100CF00065722E2E2E2000433E2000436C656172EB
:100D0000696E6720454550524F4D0A004C25640AD4
:100D1000005B435D005B445D005B535D005B575DC2
:100D2000005B525D0009025B00030100A0FA0904A8
:100D3000000001030101000921110100012240000E
:100D400007058103080001090401000103000000F8
:100D50000921110100012232000705820320000150
:100D60000904020002030000000921110100012210
:100D7000220007058303200001070503032000016B
:100D80001201000200000008EDFE00000100010257
:100D900000010E03410062006100630075007300F2
:100DA000000014036E00690063006B006F006C00AC
:100DB000610069006A0000000403090411241FBED9
:100DC000CFEFDAE0DEBFCDBF04B603FE18C08091DE
:100DD0005C0390915D03A0915E03B0915F03873047
:100DE000904BA740B04B59F410925C0310925D03F6
:100DF00010925E0310925F03E0E0F8E3099512E0C1
:100E0000A0E0B1E0E8EAFFE502C005900D92A2354E
:100E1000B107D9F723E0A2E5B2E001C01D92AC35DD
:100E2000B207E1F70E9428270C94BC2F0C94000015
:100E3000FF93EF93E0915202F0915302309709F043
:100E40000995EF91FF910895FC018591803011F093
:100E5000EFDFFBCF0895FF27E0E230E247FF0CC051
:100E6000419597FF09C0EDE260957095809590954A
:100E7000611D711D811D911D27FF02C0219530E369
:100E800050E2AA27660F771F881F991FAA1FA41771
:100E900010F0A41B63955A95A9F7AA3008F0A95F32
:100EA000A05DAF93F395611571058105910541F73B
:100EB000ED3211F4EF93F395F21718F43F93F39595
:100EC000FBCF8F91B5DFFA95E1F70895E991F9919C
:100ED0008591803021F0853219F0AADFF9CF08958D
:100EE00020E0E89455915532C1F3503311F46894E1
:100EF00055915A3348F4505390F3220F022E220F8B
:100F0000220F200D250FF4CF0EF421958991999190
:100F1000533619F3533729F1533559F1BC0188275A
:100F20009927E8945C3621F48991999168945591B8
:100F3000543639F446EF7EF077FF0DC08FEF9FEF08
:100F40000AC055374AE039F0583540E121F05236B1
:100F500042E009F00895FF93EF937DDFEF91FF9159
:100F6000B7CFFF93EF93FC0181918030B9F360DF3D
:100F7000FBCFFF93EF9368DFF1CFDF93CF93CDB734
:100F8000DEB72596A3DFCF91DF910895E8EDF0E07D
:100F900080818E7F80831092E2001092DA0010929E
:100FA000E100A0EEB0E08C9181608C9380818F771E
:100FB000808319BCA7EDB0E08C918E7F8C938081EB
:100FC0008F7E808310923E0308952091E40030913B
:100FD000E50095E6A9012091EC00822F817020FFA9
:100FE00006C08091E80080FF06C080E0089520914F
:100FF000E80022FD1AC080914B03882389F08530D8
:1010000089F08091EB0085FD0FC02091E4003091C4
:10101000E50042175307F9F29150E1F684E0089594
:1010200082E0089583E0089581E00895EF92FF92B1
:101030000F931F93CF937C018B010E94E507C82F6C
:10104000811117C08091E80085FD0BC08091E800F8
:101050008E778093E8000E94E507882399F3C82FD4
:1010600008C0F70181917F018093F10001501109BF
:1010700049F78C2FCF911F910F91FF90EF9008951A
:1010800080914D0387FF13C08091E80082FF06C066
:101090008091E8008B778093E80004C080914B0337
:1010A0008111F2CF089580914B038823D9F3809169
:1010B000E80080FFF8CF8091E8008E77ECCF982F82
:1010C0009093E900242F762F50E0891731F070912A
:1010D000EC002091ED005091F00021FD07C09F5FD2
:1010E000973071F78093E90081E008953091EB002B
:1010F0003E7F3093EB003091ED003D7F3093ED006B
:101100003091EB0031603093EB007093EC00209352
:10111000ED005093F0002091EE0027FDE0CF80E03D
:101120000895B0E0A0E0E7E9F8E00C94E42BC8ED06
:10113000D0E088818F7E8883E7EDF0E08081816058
:10114000808384E082BF81E080933E0388818E7F2C
:10115000888302EE10E0F80110821092DA0081EE2E
:10116000C82ED12CF601108288818F7788838881E0
:101170008068888388818F7D888319BC10924B0397
:1011800010924C0310924A031092490390EEE92EFC
:10119000F12CF70180818B7F808388818160888337
:1011A00042E060E080E00E945F08F60180818E7F6F
:1011B0008083F80180818160808380818860808362
:1011C000F70180818E7F8083888180618883CDB79D
:1011D000DEB7E8E00C94002CFC0180915303909161
:1011E000540386179707A0F06115710529F49091B3
:1011F000E8009E779093E80090E06115710551F446
:10120000911108C08091E80082FF34C080E0089509
:10121000BC01F2CF80914B038823C1F18530C1F12D
:101220008091E80083FD30C08091E80082FDEACF24
:101230008091E80080FFE1CF8091F3002091F200DF
:10124000382F6115710519F02830310558F091E0FB
:101250002830310509F090E02091E8002E772093A6
:10126000E800CBCF81918093F100615071092F5F2D
:101270003F4FE7CF80914B03882341F0853041F009
:101280008091E80083FFBECF81E0089582E0089559
:1012900083E0089508950895089580914003089586
:1012A0002FB7F894609155037091560380915703BE
:1012B000909158032FBF08952FB7F894809155034C
:1012C00090915603A0915703B09158032FBF0895F2
:1012D00020913503309136032817390771F0909328
:1012E000360380933503E0913303F0913403309754
:1012F00021F00084F185E02D0995089520913103B6
:10130000309132032817390771F09093320380939C
:101310003103E0913303F0913403309721F00680DC
:10132000F781E02D09950895E0913303F09134039E
:10133000309729F00190F081E02D0995089580E023
:101340000895FA01811101C0FB010995089580916A
:101350002203982F9E7F29F481708260809322035C
:1013600008958434E8F381708264F8CFAF92BF921D
:10137000DF92EF92FF920F931F93CF93DF93082F8B
:10138000162FE901E42FF0E0EA5DF94F611110C07A
:10139000E4915E2F4E2F4983E8835A83DF91CF91EA
:1013A0001F910F91FF90EF90DF90BF90AF90089545
:1013B000E62EF12C4491D42EE42FF0E026E0829F1B
:1013C000C00111242FEF30E0B9010E94AC2B802F17
:1013D00090E0880F991F55E5569FD001579FB00D9B
:1013E00011248A1B9B0B982F990F890F5901AE1856
:1013F000BF08AE9ED001AF9EB00DBE9EB00D1124B1
:101400005B2F189F80011124012F11275901A01A69
:10141000B10AAE9E8001AF9E100DBE9E100D11242C
:101420005901A81AB108AE9CC001AF9C900DBE9C9A
:10143000900D1124892F9927281B390B2E9FC0014D
:101440002F9F900D3E9F900D1124E92F6230710562
:10145000A1F050F46115710509F49DCF613071055B
:1014600081F0EB2F512F97CF6430710569F080F038
:101470006630710509F48FCFF4CFE42F4B2F592F2D
:101480008ACFE42F412F87CFEB2F542F492F83CFC3
:101490004B2F5D2DE12F7FCFF894E82FE295EF7071
:1014A000F0E031A1282F2F7081E090E001C0880F7B
:1014B0002A95EAF7982F9095932391A392A1892BCF
:1014C00082A3789408959091C90292FF06C0282FB4
:1014D00028712830F9F4877F846093FF06C0282F95
:1014E00028712831F1F4877E84612091CA0220FF9F
:1014F00006C0382F38713830D9F4877F816021FFDA
:1015000006C0282F28712831D1F4877E816194FD8F
:10151000877E0895282F24712430F9F68B7F886008
:10152000DCCF282F2471243101F78B7E8861DDCF39
:10153000382F3171313019F78E7F8860E0CF282F36
:101540002171213121F78E7E8861E1CF972F743090
:10155000A8F46C3098F470E02CE0929F600D711D3F
:101560001124FB0190E3899FE00DF11D1124EE0F82
:10157000FF1FE353FD4F85919491089580E090E023
:101580000895CF93DF93EC0182389105B1F108F013
:1015900040C08133910509F49DC048F58932910519
:1015A00009F48DC08A9709F49CC0C11522E5D207C1
:1015B00008F0BDC0C11531E5D30708F024C1C83E0D
:1015C000D10508F0A3C0C13ED10588F5C83AD105C0
:1015D00008F08EC0C53AD10508F0F6C0C130D1057B
:1015E00031F1209721F1C430D10508F545C085338C
:1015F000910509F45FC0C997C1F68091C902837053
:1016000009F036C18091CA0283FF11C0C9E2D0E05F
:101610000EC0833E910599F170F4803E910501F171
:10162000823E910511F68091C90282FD21C0CE0152
:10163000DF91CF910895863E910561F1873E910536
:1016400071F1843E910509F0B0CF8091CA0281FF0B
:10165000EECF8091C902C7EED0E084FD0DC0E7CF88
:101660008091C90280FD33C09091CA0290FFDFCF04
:10167000C3EED0E084FFDBCFD0E0C0E0D8CF8091D4
:10168000C90282FDF2C09091CA0290FDF1C084FFB0
:10169000CECFF2CF8091C90283FDDDCFC8CF80913C
:1016A000C90283FDE8C09091CA0291FFF0CFC4EE59
:1016B000D0E0BDCF8091C90285FFB9CFA7CF80917F
:1016C000C90285FDDBC08091CA0283FFB0CFC9E3A8
:1016D000D0E0ADCF8091C90286FFA9CFCAE2D0E0A9
:1016E000A6CF8091C90286FFA2CFC1E3D0E09FCFF1
:1016F000CF3BD10508F6C85AD0E0CC0FDD1FCD5244
:10170000DE4F0990D881C02DD46491CFC11540E53A
:10171000D40708F064C0C11580E4D80708F05CC0A5
:10172000CE019A9581159F4108F481CFA5CFC115AF
:1017300036E5D30718F5C11545E5D40708F07CC098
:10174000C11584E5D80708F072C09E0123703327C5
:101750009C2F96959695C115D34508F459C0C1E0C4
:10176000D0E002C0CC0FDD1F2A95E2F730E2939F54
:10177000C0011124C82BD92BDA6859CFC1158AE5CD
:10178000D80778F4C11529E5D20708F060C0C11563
:1017900038E5D30708F470CFDC2FCC27C06FD06AB0
:1017A00046CFCE0190568115904208F065CF8D2F1F
:1017B0008F710E94630A90E0982F882788279F7175
:1017C0009C012C2BE90141C0C55AD0E0C053DE4F2B
:1017D000C881D0E0D0642BCFDF70D06A28CFCE0193
:1017E0008370992721E030E002C0220F331F8A95D1
:1017F000E2F7C695C69580E2C89FE0011124C22B8E
:10180000D32BDD6814CFDC2FCC27C16FD06A0FCF6C
:10181000C1E0D0E002C0CC0FDD1F2A95E2F720E244
:10182000929FC0011124C82BD92BDC6800CFDC2F7C
:10183000CC27C46FD06AFBCE8C2F0E94630AC82FBE
:10184000D0E0DC2FCC27CC27DF71D062F0CE8C2FFC
:101850008F700E94630A34E0D695C7953A95E1F7F8
:10186000CF709C2FEC01D069E2CEC2EED0E0DFCE8B
:10187000C0EED0E0DCCEC6EED0E0D9CEC5E3D0E0FD
:10188000D6CE8091BB0281111092BB020895809543
:101890009091BA0298239093BA020895E6E5F2E097
:1018A0009191891303C0DF0111971C9292E0EC35EE
:1018B000F907B1F70895A6E5B2E0EFEF90E02D91BA
:1018C000821751F0EF3F19F4211101C0E92F9F5FFA
:1018D0009630A9F7EF3F09F408950E2E000CFF0B88
:1018E000EC5AFD4F828308958091AF0290917E0261
:1018F000981301C008958F5F8770FACFB0E0A0E021
:10190000E4E8FCE00C94E32B7C0100912D031091A2
:101910002E038091BC029091BD02082B192BCFE0C1
:10192000D0E0CC24C394D12CBC2EC6010C2E02C016
:10193000880F991F0A94E2F780239123892B49F499
:10194000219790F7B12C8B2DCDB7DEB7E9E00C9441
:10195000FF2BB7018C2F0E94A60A0E94C10A019793
:1019600079F3F1CFCF93DF93EC010E947E0CBE019F
:101970000E94A60A0E94C10ADF91CF910895943077
:1019800078F58C3068F5E82FF0E08CE0989FE00D5A
:10199000F11D11249E2F977083E0F695E7958A95A7
:1019A000E1F7EE0FFF1FEE0FFF1FE05AFD4F50E073
:1019B00040E080E0219130E0092E02C03695279565
:1019C0000A94E2F721703327042E01C0220F0A94F3
:1019D000EAF7822B4F5F5F4F4430510559F7089566
:1019E00080E00895943098F58C3088F5E82FF0E089
:1019F0008CE0989FE00DF11D11248E2F877041E03F
:101A000001C0440F8A95EAF783E0F695E7958A9539
:101A1000E1F7EE0FFF1FEE0FFF1FE05AFD4F30E022
:101A200020E070E05191DF011197CB01022E02C03E
:101A3000969587950A94E2F781708195852784238E
:101A400085278C932F5F3F4F2430310559F7089538
:101A5000FC0183819481892B29F0808191818923E4
:101A60008F3F51F480E00895843FE1F717C0883E2E
:101A7000A8F0813FB9F712C0808191810E94B20C19
:101A800092959F70963099F358F4925F9F709230C0
:101A900048F7803F19F040F7883E20F781E008952D
:101AA0009A5FF4CF829590E09C01220F331F220FA2
:101AB000331F2C7C95958795959587958373282B57
:101AC00030E0C901880F991F8A7A359527952575C9
:101AD000822B0895292F332740E02115310511F07D
:101AE000C90148E09C0164E0369527956A95E1F7C5
:101AF0002115310511F04C5FC9019C0136952795E0
:101B0000369527952115310511F04E5FC90196953F
:101B10008795892B09F04F5F842F08959C019A9532
:101B200081159F4140F4832F817031FD826032FF27
:101B300003C08460089580E008959FB7F8941092E0
:101B40003C039FBF90914B03943009F048C0209113
:101B5000E9002F703091EC00932F917030FD90E8E8
:101B6000922B23E02093E9002091EB0020FF34C06A
:101B70002091EE0027FF30C020913B03222321F06B
:101B80002091E80025FF28C010923B0326E0309109
:101B9000E80035FF14C08093F1008091E80085FDD6
:101BA00027C08091E80080FFFCCF8091E8008E770D
:101BB0008093E8009F709093E90080E00895309151
:101BC0004B03343049F43091EB0035FD05C0215012
:101BD00041F481E080933B039F709093E9008FEF85
:101BE0000895EFE9FFE03197F1F700C00000CFCF93
:101BF0008FB7F89421E020933C038FBFDBCF809315
:101C0000380370933A036093390380914B03843017
:101C100001F582E08093E9008FEF9091E800815018
:101C200095FD06C095ED9A95F1F700008111F5CF6D
:101C30008091E80085FF0DC050E040E063E070E077
:101C400088E393E00E9416088091E8008E778093E5
:101C5000E8000895BC0184E00E94FF0D0895BC01D6
:101C600083E00E94FF0D0895CF93DF93EC0181E0A4
:101C70008093E9008FEF9091E800815095FD06C0B8
:101C800095ED9A95F1F700008111F5CF8091E8006C
:101C900085FF14C050E040E068E070E0CE010E9493
:101CA00016088091E8008E778093E80088E0FE01B6
:101CB000A1E4B3E001900D928A95E1F7DF91CF9115
:101CC00008958091220380FD0AC0EFEEF2E01182B8
:101CD00010821282339653E0E232F507C1F7519A2F
:101CE0003BB13D7F2BB122604FB7F8948FEE92E06D
:101CF000FC015191CF0168E02BB9000000C057FFF3
:101D00003BB9550F000000C000C000C03BB900C087
:101D10006A9591F7F3E082329F0751F74FBF8FE545
:101D200094E00197F1F700C0000008950F931F930E
:101D3000CF93DF93CFEED2E0FE01118210821282A8
:101D4000339683E0E232F807C1F710E000E08091BB
:101D5000EE02082E000C990B081719078CF18091E0
:101D60001801082E000C990B801791074CF19E0169
:101D70004091250360912403809123030E94B609BA
:101D80000F5F1F4F23960131110509F70E94610E65
:101D9000809117019091EE02980F9093EE0220919E
:101DA0001801280F20931801121614F490311CF01A
:101DB000819580931701DF91CF911F910F91089525
:101DC000198218821A82DCCFB0E0A0E0EAEEFEE0D1
:101DD0000C94E32BFC018281DD24DA9480FD02C0A7
:101DE000DD24D3940FEE12E0D0E0C0E021E1B22E6A
:101DF000F80111821082128294E0E92EF12CC12C9C
:101E00008091ED028C0D8231C4F16B2D0E949E2BCE
:101E1000892F082E000C990B8C179D0791F4809147
:101E200025038E9DA0018F9D500D1124559547953A
:101E300055954795980160912403809123030E9452
:101E4000B609CD0CF1E0EF1AF108D1F621960D5F3D
:101E50001F4FC131D10561F60E94610E8091ED02E4
:101E600091E0D91210C081110CC080E18093ED0285
:101E7000CDB7DEB7E9E00C94FF2B87FFCACF8F5EAA
:101E8000C8CF8150F3CF90E00196BE010E94C02BD5
:101E9000EDCFEF92FF921F93CF93DF93EC018FEE84
:101EA000E82E82E0F82E10E08C8197014091250306
:101EB00060912403810F0E94B609115F83E0E80E50
:101EC000F11C1F3F89F70E94610E9A818C8190FF5F
:101ED00008C08F5F8C83DF91CF911F91FF90EF90AF
:101EE00008958150F7CF9091220390FF0CC0EFEE40
:101EF000F2E0818360834283339693E0E232F90714
:101F0000C1F70E94610E0895A3E0B0E0EAE8FFE0A7
:101F10000C94EA2B9091220390FF0AC09E012F5F40
:101F20003F4F0E94B6094B8169818A810E94730FDD
:101F30002396E2E00C94062CCF93DF93EC01E2E2CF
:101F4000F3E0438162818C810E94840F8C818F5FDA
:101F50008C83DF91CF9108951092EC0280912C0335
:101F600080FF08C081EF97E09F938F930E94BD0789
:101F70000F900F900895CF9384E090E00E94112C71
:101F8000C82F82E290E00E94112C982F8C2FCF91C5
:101F9000089580932703682F8CE090E00E94252C01
:101FA00080912C0380FF0EC0809127031F928F9396
:101FB0008AE098E09F938F930E94BD070F900F9047
:101FC0000F900F900895CF93DF93EC016C8170E038
:101FD00090E080E00E94A32D20E030E04FE753E442
:101FE0000E94C62C2BED3FE049E450E40E94CC2E29
:101FF0000E94392F0E94402D2BE43AE34EE25FE32A
:102000000E94592C20EF3BEF48ED52E40E94CC2E69
:102010000E94722D462FE2E2F3E0628181810E94EC
:10202000840F8C818F5F8C83DF91CF9108956091B5
:102030002203669570E04BE050E08CE091E00E9456
:10204000A22F892B19F481E08093EC020E945C0995
:102050009093E6028093E50280912C0380FF08C0F4
:1020600088ED97E09F938F930E94BD070F900F908C
:102070000895CF92DF92EF92FF926B017C010E9454
:10208000A709B701A60188E090E00E94372CFF90D5
:10209000EF90DF90CF900895A7E0B0E0E2E5F0E1A7
:1020A0000C94DA2B582E262E342E2F839091220357
:1020B00090FF46C0E92FE695AE2FB0E0AF5DBD4F73
:1020C0008C918093EB029E7F9230F1F59E012F5F01
:1020D0003F4F852D0E94B6094B8169818A810E94FC
:1020E000730F5092230320922403309225038F8193
:1020F000882309F48CC0609122037091230380919E
:102100002403909125030E94391080912C0380FFB5
:1021100017C0809125031F928F93809124031F92F3
:102120008F93809123031F928F9387E897E09F936B
:102130008F930E94BD070FB6F894DEBF0FBECDBFD0
:102140002796E2E10C94F62B823019F430902503A7
:10215000C8CF863019F450902303C3CF8930D9F308
:10216000883109F0BECFE8518E2F81708D838E2F7C
:10217000809581708E83E695F0E0ED52F84F949152
:102180009C83692E712C8FEEE82E82E0F82ED12CE4
:10219000C12C10E000E091E1892E912C2CEAA22EB6
:1021A00027E0B22EC601B4010E94AC2B8D81452CD4
:1021B00081112BC0460E80912C0380FF13C01F920B
:1021C0009C819F931F928E818F931F924F921F939A
:1021D0000F93BF92AF920E94BD070FB6F894DEBF77
:1021E0000FBECDBF9701432D622D842D0E94B609ED
:1021F0000F5F1F4FC60CD71C93E0E90EF11C013195
:10220000110581F60E94610E6CCF461AD4CF8091E1
:102210002C0380FF95CF1F923F921F922F921F9207
:102220005F9280E697E083CFE2E2F3E0438128E02B
:10223000421B08F440E021E0628181810E944C1041
:102240000895E2E2F3E0438128E0420F08F44FEF03
:1022500021E0628181810E944C100895E2E2F3E066
:10226000628128E0621B08F460E021E04381818103
:102270000E944C100895E2E2F3E0628128E0620FD0
:1022800008F46FEF21E0438181810E944C10089592
:10229000E2E2F3E0818121E04381628188500E9483
:1022A0004C100895E2E2F3E0818121E043816281F4
:1022B000885F0E944C10089580912603882319F0AE
:1022C00081508093260360912203709123038091B3
:1022D0002403909125030E943910089580912603CC
:1022E000833018F48F5F80932603609122037091EE
:1022F000230380912403909125030E9439100895AF
:102300009091220390FF40C0917081113EC0926075
:1023100090932203662309F43FC0609122037091D9
:10232000230380912403909125030E94391080910A
:102330002C0380FF0FC08091220386951F928F93FC
:1023400084E497E09F938F930E94BD070F900F90B6
:102350000F900F9060912203669570E04BE050E083
:102360008CE091E00E94A22F892B11F10E94AC0F0A
:1023700081E08093E80220E04091250360912403EE
:10238000809123030E944C100895823210F09264D1
:10239000BFCF880F982BBCCF80912C0380FFDACF62
:1023A0008091220386951F928F9386E297E0CACF91
:1023B0000E941710DDCF809122038695815009F489
:1023C00081E261E00E948011089580912203869548
:1023D0008F5F823208F081E061E00E9480110895F1
:1023E0009091220390FF08C09695981728F09617B1
:1023F00018F40E94E511089561E00E94801108958B
:10240000E2E2F3E083E0808311828FEF82838383B3
:10241000148260817181828193810E9439100895B4
:102420000F931F93CF93DF938091BA029091B902DB
:10243000892B809354029091BB02992391F0892BB0
:102440008093540220E086E592E0FC013191CF01B7
:1024500031112F5FF2E08C359F07B9F721110E94EF
:10246000410C48E050E061EB72E084E592E00E94AC
:10247000AF2F892B09F441C088E0E4E5F2E0A1EB3D
:10248000B2E001900D928A95E1F7E0913303F0916B
:102490003403309791F10280F381E02D84E592E0DE
:1024A000099580912C0382FF28C080FF04C08BEB2C
:1024B00092E00E942407D0E0C0E005EB12E080919A
:1024C0002C0380FF0EC0FE01EC5AFD4F80811F924D
:1024D0008F931F930F930E94BD070F900F900F9043
:1024E0000F902196C830D10551F780912C0380FFC1
:1024F00004C083EB92E00E942407DF91CF911F91EB
:102500000F91089590E080E00E947E0990E080E0C5
:102510000E9468091092B9020E94101208959093C7
:102520002E0380932D030E948212089521E030E053
:1025300002C0220F331F8A95E2F7209530958091D3
:102540002D0390912E03822393230E948F120895CE
:102550009091B002809589238093B002282F277034
:1025600091F4282F082E000C330B9217130659F004
:102570009091CA0292FF07C08595859585950E9426
:1025800096121092B0020895CF93DF93D82FC09186
:10259000CA02C2FB882780F98D1711F1D0FBC2F95E
:1025A000C093CA026091C90284E090E00E94252C89
:1025B0006C2F82E290E00E94252C82E00E94A812FB
:1025C00080912C0380FF0CC01F92DF938EE992E074
:1025D0009F938F930E94BD070F900F900F900F90C5
:1025E000DF91CF91089521E030E002C0220F331F28
:1025F0008A95E2F780912D0390912E03822B932BE5
:102600000E948F1208959093BD028093BC020E9495
:10261000821208951092BA02E6E5F2E086E0DF0148
:102620001D928A95E9F70E9482120895AAE2B0E00D
:10263000ECE1F3E10C94E92B8DE493E02091F100BF
:10264000DC012D93CD01B3E085359B07B9F780916F
:102650004E03833009F470C0B8F4813009F447C0E8
:10266000823009F4B1C08091E80083FF84C2809178
:102670004D0390914E039A3008F07DC2E92FF0E0AF
:10268000E254F04D0C94D42B8A3009F48CC08B307A
:1026900009F46FC0893039F780914D03813219F701
:1026A00080915103909152030297E8F68091E800DF
:1026B000877F8093E8008091E80082FF38C0909186
:1026C000F3008091F200029731F48091F1008130A3
:1026D00011F0863021F48091F100809340038091C5
:1026E000E8008B778093E8000E944008BCCF80917F
:1026F0004D03813A09F0B7CF8091E800877F80933E
:10270000E8008091510390915203892B61F468E0B5
:1027100081E493E070E00E94EC088091E8008B7700
:102720008093E800A0CF60E090E080E0F3CF80915C
:102730004B038111C0CF97CF80914D03813A09F0AF
:1027400092CF8091510390915203892B09F08BCF46
:102750008091E800877F8093E8008091E80080FF07
:10276000FCCF809119018093F1008091E8008E7771
:10277000B9CF80914D03813209F075CF809151031B
:1027800090915203892B09F06ECF8091E800877FEA
:102790008093E8000E94400880914F0380931901C4
:1027A0000E940A1360CF80914D03813209F05BCF04
:1027B0008091E800877F8093E8000E944008809124
:1027C000500380933F034FCF80914D03813A09F02E
:1027D0004ACF8091E800877F8093E8008091E800ED
:1027E00080FFFCCF80913F03BECF803899F08238C4
:1027F00009F0C1C1809151038F70873008F0BBC1CF
:102800008093E9008091EB0085FB882780F9109286
:10281000E90006C08091490390914A0391118260BA
:102820009091E800977F9093E8008093F1001092D8
:10283000F1008091E8008E779AC1882309F488C15D
:10284000823009F098C180914F0381118BC1809132
:1028500051038F702FEF280F263008F08CC1809322
:10286000E9002091EB0020FF7DC1933031F480918D
:10287000EB0080628093EB0075C19091EB0090615A
:102880009093EB0021E030E001C0220F8A95EAF737
:102890002093EA001092EA008091EB008860EACF72
:1028A000811169C110914F031F778091E3008078F7
:1028B000812B8093E3008091E800877F8093E8007C
:1028C0000E9440088091E80080FFFCCF8091E300E7
:1028D00080688093E30082E0111183E080934B03D2
:1028E0004AC18058823008F046C120914F03309190
:1028F00050032C3DE3E03E07A1F583E08A838AE2A2
:1029000089834FB7F894DE01139620E03EE051E250
:10291000E32FF0E050935700E49120FF03C0E295CD
:10292000EF703F5FEF708E2F90E0EA30C0F0C796F7
:102930008D939D932F5F243159F74FBF8091E8000D
:10294000877F8093E8006AE270E0CE0101960E94E2
:10295000EC088091E8008B778093E8000CC1C0966A
:10296000E7CF8091510390915203432F5527433075
:10297000510509F44AC078F54130510509F47AC08F
:102980008BE590E0E5E2FDE04230510509F0F3C04F
:102990002091E800277F2093E80020915303309195
:1029A00054038217930708F49C0140E02115310578
:1029B00009F065C0411163C08091E80082FDC9CF74
:1029C00080914B03882329F2853019F28091E80029
:1029D00083FFF2CFBECF4132510509F43CC04232F1
:1029E000510509F0C8C08330910508F0C4C0FC014E
:1029F000EE0FFF1FEA5BFD4F0190F081E02D8D5B34
:102A00009D4FDC018C9190E01AC0332721303105B5
:102A1000D1F02115310561F02230310509F0ABC04C
:102A2000E2E9FDE0E4918E2F90E0E2E9FDE007C0ED
:102A3000E8EBFDE0E4918E2F90E0E8EBFDE00097FD
:102A400009F499C0A5CFE2EAFDE0E4918E2F90E071
:102A5000E2EAFDE0F4CF8330910508F08CC0880FE6
:102A6000991FFC01E45BFD4F0190F081E02D89E0AE
:102A700090E08ECF82E190E0E0E8FDE089CF8091A8
:102A80004B03882309F465CF853009F462CF809128
:102A9000E80083FD5ECF8091E80082FD8DCF8091BC
:102AA000E80080FF83CF9091F3008091F200211520
:102AB000310519F08830910550F041E0089709F090
:102AC00040E08091E8008E778093E8006FCF4491DA
:102AD0004093F1003196215031090196E8CF8038BA
:102AE00009F049C08091E800877F8093E8008091D9
:102AF0004C038093F1009DCE81113DC010914F0396
:102B00001230C8F58091E800877F8093E800109329
:102B10004C030E944008112311F084E005C080910D
:102B2000E30087FDFACF81E080934B0342E061EC44
:102B300081E00E945F0842E261EC82E00E945F084F
:102B400042E261EC83E00E945F0880914B0313C076
:102B500080914F03813079F481E0933009F080E077
:102B600080934A031092E9008091E800877F809368
:102B7000E8000E9440088091E80083FF0AC080912D
:102B8000E800877F8093E8008091EB00806280936B
:102B9000EB00AA96E3E00C94052CCF93C82F1F926C
:102BA0008F938CE09DE09F938F930E94BD0781E0FF
:102BB00090E002C0880F991FCA95E2F70E940313A4
:102BC0000E940A130F900F900F900F90CF910895CD
:102BD0000E940A132FEF84E39CE021508040904034
:102BE000E1F700C0000081E08093E00080E2809384
:102BF000D8001092C9008FE19EE40197F1F700C060
:102C0000000087E090EBDC0180935C0390935D0310
:102C1000A0935E03B0935F0388E19CE00FB6F89445
:102C2000A895809360000FBE90936000FFCF0E9434
:102C30000A132FEF84E39CE0215080409040E1F79D
:102C400000C0000088E19CE00FB6F894A89580933E
:102C500060000FBE90936000FFCF882341F0809505
:102C60009091B90289238093B9020E9410120895AD
:102C7000882339F09091B902982B9093B9020E9461
:102C800010120895882321F00E94470C0E94101210
:102C90000895882339F09091BA02982B9093BA0244
:102CA0000E9410120895882309F44DC0823879F4E7
:102CB0000E94940981FF47C089E30E945B0C0E9437
:102CC000101289E30E944E0C0E941012089583385E
:102CD00059F40E94940980FF36C083E50E945B0C82
:102CE0000E94101283E5EECF843859F40E949409B3
:102CF00082FF29C087E40E945B0C0E94101287E4C7
:102D0000E1CF9CEF980F913AE8F290E2980F98305B
:102D100050F4877091E001C0990F8A95EAF7892FE6
:102D20000E94470CD1CF9BE5980F933028F490E098
:102D300080E00E947E090895885A873120F490E04F
:102D400080E00E9468090895A8E0B0E0EAEAF6E1B0
:102D50000C94DE2B8E010F5F1F4F88E0F80111925B
:102D60008A95E9F791E0E92E92E0F92E680125E0D5
:102D7000622E22E0722E88248394912CF701819197
:102D80007F018F3F09F446C0F894E82FE295EF7079
:102D9000F0E021A18F70A40102C0440F551F8A9555
:102DA000E2F7CA01922F982B91A392A180958923D3
:102DB00082A3789400C0E5E0F2E021E030E0B12C9D
:102DC000A12C41914F3F09F471C0A42FA295AF707F
:102DD000B0E090968C9190E04F7002C095958795E9
:102DE0004A95E2F780FD62C0C901A82AB92A220FDC
:102DF000331F52E0E131F50721F7F7013197808168
:102E00008F3F11F00E944C0A80EA8A95F1F7F60193
:102E1000B182A082F2E0CF0ED11C6E147F0409F0C3
:102E2000ADCF48E050E0B80181EC92E00E94AF2FB6
:102E3000892B09F43EC088E0F801A1ECB2E00190D2
:102E40000D928A95E1F781E08093C0020E945C09AF
:102E50009093BF028093BE022091BE023091BF02C8
:102E60004FB7F8948091550390915603A091570362
:102E7000B09158034FBF821B930B0597F0F048E0C9
:102E800050E061EC72E080ED92E00E94AF2F892B60
:102E9000C9F088E0E1ECF2E0A0EDB2E001900D9223
:102EA0008A95E1F781E01092C00208C090E080E0CE
:102EB0009CCF8091C0028111CFCF80E02896EEE0B8
:102EC0000C94FA2B80E0EFCF68EE7EEF90E080E08C
:102ED0000E94432C60E082E090E00E94252C60E09C
:102EE00083E090E00E94252C1092BD021092BC025B
:102EF00060E084E090E00E94252C64E082E290E0B3
:102F00000E94252C60E085E090E00E94252C60E086
:102F100086E090E00E94252C6FEF87E090E00E9411
:102F2000252C40E050E0BA0188E090E00E94372C68
:102F300060E08DE090E00E94252C40E050E0BA0176
:102F400088E190E00E94372C60E087E190E00E94E9
:102F5000252C40E050E0BA018CE190E00E94372C33
:102F600070E060E080E290E00E94432C40E050E09E
:102F7000BA0188E190E00E94372C40E050E0BA01AD
:102F80008FE090E00E94372C40E050E0BA0183E1EE
:102F900090E00E94372C0895EF92FF920F931F93B9
:102FA000CF93DF938B3109F413C108F0B4C08B3099
:102FB00009F4CFC008F086C0863009F4DDC048F4BB
:102FC000853009F4B6C08DE69CE00E94240780E0BD
:102FD000E3C0873009F4E5C08830A9F783E090E0CA
:102FE0000E94112C1F928F9381E29AE09F938F93FE
:102FF0000E94BD0782E090E00E94112C83FB99277C
:1030000090F91F929F9382FB992790F91F929F93AB
:1030100081FB992790F91F929F93982F91701F928F
:103020009F931F928F9388ED99E09F938F930E94B7
:10303000BD070E94BB0F93FB222720F91F922F93FD
:1030400087FB222720F91F922F9386FB222720F946
:103050001F922F9385FB222720F91F922F9384FB29
:10306000222720F91F922F9383FB222720F91F92FA
:103070002F9382FB222720F91F922F9391FB222767
:1030800020F91F922F93292F21701F922F9381FBDC
:10309000222720F91F922F93282F21701F922F9300
:1030A0009F938F9389ED98E09F938F930E94BD0724
:1030B0008DB79EB78A960FB6F8949EBF0FBE8DBF90
:1030C00081E06AC0803109F49BC080F48E3009F041
:1030D0007ACF90912C03892F8B7F92FF846080930D
:1030E0002C0382FF8AC088E99CE07EC0863109F407
:1030F00097C0893109F067CF8AE191E09F938F9360
:103100008FEF9BE09F938F930E94BD070F900F90CE
:103110000F900F90D5CF8A3241F188F4873209F1B0
:1031200028F48E3108F44FCF8D511CC0893209F03C
:103130004ACF8BED9CE00E9424070E94E81583345F
:1031400068F48A3308F091C0853359F0883309F068
:103150003ACF8EE39AE00E942407B2CF833409F07D
:1031600032CF80E00E94CD15ABCF8BEF9CE00E9468
:1031700024070E946417A4CF80912C03807F809342
:103180002C0384EE9BE00E94240787EF9CE00E94C2
:10319000240781E080932B03CDB7DEB7E6E00C94E3
:1031A000022C90912C03892F8E7F90FF8160809359
:1031B0002C0380FF03C08FEC9CE0CDCF82EC9CE021
:1031C0000E94240780912C03817F80932C0378CF69
:1031D00090912C03892F8D7F91FF826080932C0327
:1031E00081FF08C085EB9CE00E94240780912C039E
:1031F0008160EBCF87EA9CE0AECF88E89CE0ABCF64
:1032000090912C03892F877F93FF886080932C03F4
:1032100083FF03C08CE79CE0E7CF8FE69CE09BCF69
:103220000E945009162F072FF82EE92ED0913F0348
:10323000C09119010E949409EF92FF920F931F937E
:103240001F92DF931F92CF931F928F9382E09CE097
:103250009F938F930E94BD078DB79EB70C960FB6B4
:10326000F8949EBF0FBE8DBF2BCF89537BCFCF93DA
:10327000C82F8823C9F08238C9F40E94940981FDBF
:1032800013C089E30E945B0C0E9410122FEF87EE9F
:1032900093E0215080409040E1F700C0000089E3B6
:1032A0000E944E0C0E941012CF9108958338A1F411
:1032B0000E94940980FDF8CF83E50E945B0C0E9478
:1032C00010122FEF81EE94E0215080409040E1F702
:1032D00000C0000083E5E4CF8438A1F40E94940983
:1032E00082FDE2CF87E40E945B0C0E9410122FEF58
:1032F00081EE94E0215080409040E1F700C0000052
:1033000087E4CECF8CEF8C0F813A08F042C08091D9
:103310002B03882399F08130D9F010922B03E6E536
:10332000F2E08CE592E02191C21709F45EC08E179D
:103330009F07C9F78C2F0E945B0CB4CF8091BA0213
:10334000823269F78C2F0E94CC178111ADCFE7CF65
:103350008091BA028232B1F3C431B9F038F4CB3083
:1033600049F088E992E00E94240711C0C93269F04F
:10337000C833B9F784EE9BE00E9424078AE992E003
:103380000E94240781E08170E0CF10922B0380E03F
:10339000FACF80E28C0F883068F4C77021E030E00B
:1033A00001C0220FCA95EAF78091BA02822B80935E
:1033B000BA0278CFEBE5EC0FE33040F4F0E0E053F5
:1033C000FE4F808190E00E947E096ECFC85AC731BF
:1033D00008F06ACFEC2FF0E0EE0FFF1FED52FE4F2A
:1033E000808191810E9468095FCF8C2F0E944E0CD2
:1033F0000E9410129FCF1F93CF93DF93182FD0E01E
:10340000C0E0893311F4C0E5D0E0812F0E94371964
:10341000209739F4812F0E945316DF91CF911F918D
:1034200008958FE99FE00197F1F700C00000219710
:10343000EFCF0F931F93CF93DF93C62FD42F022F7D
:10344000FC0182818823A9F060935B030E945C09E0
:1034500090935A0380935903C77081E001C0880F8D
:10346000CA95EAF70E944916DF91CF911F910F91FB
:10347000089580915B0368133DC0209159033091FA
:103480005A034FB7F8948091550390915603A09139
:103490005703B09158034FBF821B930B883C910593
:1034A00048F510E21D0F6D17B9F080E2860F8830E5
:1034B00040F4C77081E001C0880FCA95EAF70E9406
:1034C0004216183048F481E09D2F977001C0880F94
:1034D0009A95EAF70E944916802F0E94FB1918302E
:1034E00018F6D77081E001C0880FDA95EAF70E94DC
:1034F0004216BACFC77081E001C0880FCA95EAF7BB
:10350000F6CFB0E0A0E0E7E8FAE10C94E52BE82F75
:10351000F0E0E75AF74FD490282F26952695269568
:1035200030E0F901E75BF74F0491877010E0082E57
:1035300002C0159507950A94E2F701701127F90169
:10354000E75CF74FE490F12C082E02C0F594E79465
:103550000A94E2F791E0E922FF24F901E75DF74FD1
:10356000C491D0E002C0D595C7958A95E2F7C170A5
:10357000DD270115110519F081EE0E943719E114BC
:10358000F10419F086EE0E9437198D2D0E94FB1967
:10359000E114F10419F086EE0E945316011511058D
:1035A00019F081EE0E945316CD2B19F08CE20E9487
:1035B000FB19CDB7DEB7E7E00C94012C90912703FF
:1035C000923071F48A3050F490E009966AE070E02D
:1035D0000E94C02B875A0E94FB1908958650FBCF8A
:1035E00096EF980F963020F0805D0E94811A089522
:1035F000895AFBCFB0E0A0E0E0E0FBE10C94E32BC4
:103600006B017C01C7E0D0E00CE110E0BB24B39477
:10361000D701C601002E04C0B695A795979587954A
:103620000A94D2F78F70A1F4B11002C00E94DE1A82
:10363000219704501109CF3FDC0729F4CDB7DEB73D
:10364000E9E00C94FF2BC430D10514F7B12CE0CF86
:103650000E94DE1AB12CECCFCF92DF92EF92FF9254
:103660000F931F93CF938C017B016C0180EEC81ADE
:10367000D108C8010E948E0DC82F98E0C916D10448
:10368000D0F40E944916802F0E943719E114F104EA
:10369000A9F4802F0E94531688E0C816D104C0F404
:1036A0008C2F0E944216CF911F910F91FF90EF90A7
:1036B000DF90CF9008950E943816E5CF8FE99FE004
:1036C0000197F1F700C0000091E0E91AF108DECFA0
:1036D0008C2F0E942D16E7CF99B1292F217090953C
:1036E00091709093300330912F03931302C088237D
:1036F00091F021110CC080912D0390912E030E9416
:103700006A0D813081F0882339F0823081F0809118
:10371000300380932F03089570E060E089E091E02A
:103720000E942C1BF4CF88EA0E94FB19F0CF8EEA8E
:10373000FBCFA5E0B0E0EFE9FBE10C94E02B7C01CE
:10374000FC0183819481892B31F0808191818923CF
:103750008F3F09F079C62596ECE00C94FC2B0E9473
:103760007E0C182F682F89819A810E94F20C698142
:103770007A81812F0E94A60A8C01F7018281023B87
:10378000FDE51F0709F41BC1033B2DE5120709F4F2
:103790007FC1F7018281882389F0043EFCE51F0781
:1037A00009F492C108F07EC1023E3CE5130709F41A
:1037B00087C1033E8CE5180709F484C117FFF1C1E6
:1037C000F7018281882309F4AAC068010115F0EC91
:1037D0001F0708F47FC120ECD21A8091B9029091A2
:1037E000BA02892B9091BB02892B8272BB24B394BD
:1037F000811101C0B12C0E94940986958170B81680
:1038000029F0CC0CCD2CCC1CDD08D194E894C7F861
:10381000DD24F601EE0FFF1FEE0FFF1FE955FE4FEF
:1038200085909590A590B4908114910481E1A806AB
:10383000B10408F074C08114910491E0A906B104A8
:1038400028F080912703823009F469C00E9494090E
:103850008695817080935E020E94940981708093A6
:103860005D0280912703813039F480915E028823C4
:1038700019F089E30E94FB198091BA0280935C02DF
:103880001092BA021092B90280912703823009F493
:1038900045C108F022C1882309F435C1813009F4FB
:1038A00036C18FE39CE90197F1F700C00000811455
:1038B000910491E0A906B10408F449C1809127035D
:1038C000811145C1E1E0AE1AB108C501B4014AE079
:1038D00096958795779567954A95D1F778528F4F4A
:1038E0009F4F0E94FA1AF3E09F22AA24BB24C5012D
:1038F000B40174528F4F9F4F0E94FA1A8091270390
:10390000823009F443C108F025C1882309F42EC18F
:10391000813009F42FC180915C028093BA02F701D3
:103920008281882309F4A1C510925B030430FDE570
:103930001F0708F081C10B3F2CE5120730F4C801C6
:1039400082509C45449708F082C10E94BB0F90931F
:10395000CA028093C9020231ECE51E0709F480C255
:1039600008F0CCC109302CE5120709F457C208F061
:1039700096C105308CE5180709F440C208F082C1F1
:103980000330ECE51E0709F431C208F033C2809120
:10399000C902816002302CE5120709F4ACC16091C4
:1039A000C9021091CA0284E090E00E94252C612F88
:1039B00082E290E00E94252C0E940A1318C18823FD
:1039C00009F462C076E8A72E71E0B72EEAE09E2ED9
:1039D000F5018491882309F4DCCE813009F050C0D0
:1039E0006501FFEFCF1ADF0AF6018491813069F497
:1039F0006501F2E0CF0ED11CF60184910E94FB1903
:103A000056012FEFA21AB20AE3CF823049F46501C2
:103A1000F2E0CF0ED11CF60184910E943719F0CF4D
:103A2000833049F46501F2E0CF0ED11CF601849198
:103A30000E945316E5CF843019F76501F2E0CF0EEE
:103A4000D11CF601249190E080E0F60131962053DC
:103A5000330B2A30310548F0019790F2EFE9FFE08F
:103A60003197F1F700C00000F7CF989EA001999E12
:103A7000500D1124C901840F951F24916F01E5CFCA
:103A80000E94811A6501BCCF88E20E94FB1981CE99
:103A9000882309F47ECE70E060E08BE294E00E941F
:103AA0002C1B77CE063E9CE5190791F078F085E057
:103AB000013BFDE51F0709F081CE0E94C90F7ECEB4
:103AC00080E0FBCF81E0F9CF82E0F7CF83E0F5CF54
:103AD00084E0F3CF30E8D31A9CCE843099F185305E
:103AE00009F0DFCE70E060E08BE191E00E942C1BDA
:103AF00070E060E085E290E00E942C1B70E060E0E6
:103B000088E290E008C082EE0E943719CACE70E0C9
:103B100060E088E193E00E942C1BC3CE80915D029F
:103B2000811103C083E50E94FB1982EE0E943719C0
:103B3000EFE3FCE93197F1F700C0000087E50E9450
:103B4000FB19AFCE86EE0E94FB1988E1F8CFC501C4
:103B5000B401D2CE843019F1853009F0DCCE70E0AA
:103B600060E088E290E00E942C1BD5CE82EE0E949D
:103B70005316D1CE8CE20E94FB1980915E028823FD
:103B800009F4C9CE89E30E94FB19C5CE82EE0E94DA
:103B9000531680915D028111BECE83E5F4CF88E299
:103BA000F2CF043F2CE51207C1F188F4093D8CE502
:103BB000180779F10A3D9CE51907D9F1083DECE5B4
:103BC0001E0709F0ACCE26E241EE61EE0DC0063FC5
:103BD000FCE51F0751F128F127E245EE66EE073FAD
:103BE0003CE5130709F09BCEC7010E94191A80918A
:103BF000B002877009F4AFCDF7018281882309F400
:103C0000AACD8091CA0282FFA6CD82E00E94A812AE
:103C1000A2CD27E245EE65EEE7CF26E241EE60EE6B
:103C2000E3CF27E245EE64EEDFCF26E241EE62EE1F
:103C3000DBCF28E241E0EFCF063A3DE5130709F478
:103C400084CED0F402369DE5190709F47ECE063104
:103C50008CE5180709F015C48091BA028A7A91E0C0
:103C600009F490E090935F02811124C189E20E94DF
:103C70005B0C0E941012BBCFC8018E5A9D45039762
:103C800030F763CE8091C902806207303CE51307AC
:103C900091F108F4BFC08091C90280642CC00D303E
:103CA0009CE5190709F4C4C090F48091C9028E7F85
:103CB0000B30FCE51F07F9F08091C9028C600C30D5
:103CC0002CE51207C0F08091C9028D7F14C00F301F
:103CD0003CE5130709F4BCC008F4AEC000319CE514
:103CE000190709F4B9C08091C9028F7B0131ECE555
:103CF0001E0709F054CE8093C90251CE0115FDE58F
:103D00001F0709F4B7C0A8F50B3F3CE5130709F4FA
:103D100079C0C0F404319CE5190709F4B9C008F46E
:103D2000A5C00531FCE51F0709F039CE8091C90215
:103D300082FB992790F921E0922790FB82F990FB72
:103D400083F9D9CF0D3F2CE5120709F479C008F4A7
:103D50005DC00E3F8CE5180709F476C08091CA0259
:103D600083600F3F9CE5190709F019CE8093CA02C2
:103D700016CE0236EDE51E0709F495C090F4023028
:103D80002DE5120709F48DC008F478C060E0033017
:103D90008DE5180709F003CE8EE090E00E94252CF7
:103DA000FECD0E3A9DE51907E9F060F49091C90245
:103DB000892F8E7F90FF8160063AFDE51F0709F489
:103DC0009ACFEDCD0F3A2DE5120771F1003B3DE59D
:103DD000130709F0E4CD9091CA02892F877F93FFE2
:103DE0008860C4CF8091CA028860C0CF8091C90228
:103DF000826081CF8091C90284607DCF8091C902A9
:103E0000886079CF8091CA028160B0CF8091CA0268
:103E10008260ACCF8091C90280616DCF0E940A138D
:103E20008091C902806867CF8091CA02877F9ECF48
:103E30008091C9028B7F5FCF8091C902877F5BCF62
:103E40008091CA028E7F92CF8091CA028D7F8ECFE1
:103E50008091C9028F7E4FCF8091C9028F7D4BCF59
:103E60000E940A138091C9028F7745CF8091C902C1
:103E7000837F41CF8091CA028C7F78CF8091CA0224
